:10000000D7EF03F00000000000EF00F00000000058
:0A0010000000000000000000F3D71C
:0C001C0072B201D0FDD7E1C073FF1200EA
:0E002800ACB202D00000FCD7E1C0ADFF120068
:100036000001E151030A00E1E151040A00E1E15146
:0C004600050A00E1E151060A00E1120089
:10005200F250026EF29E0500FF6A0150FE6E0050E1
:08006200FD6E02BEF28E1200D9
:04006A006B84120091
:10006E0015C0DDF016C0DEF017C0DFF018C0E0F0EE
:10007E00C582C5A21FD0155016101710181019E002
:10008E000001DD51DE11DF11E0110CE123C0E1FFB3
:10009E0024C0E2FF060EE66E21C000F022C001F081
:1000AE00D1DF08D0010E0001DD5F000EDE5BDF5BED
:0600BE00E05BDFD7120039
:1000C40019C0DDF01AC0DEF01BC0DFF01CC0E0F088
:1000D4006B826BA21FD019501A101B101C1019E050
:1000E4000001DD51DE11DF11E0110CE127C0E1FF59
:1000F40028C0E2FF060EE66E25C000F026C001F01F
:10010400A6DF08D0010E0001DD5F000EDE5BDF5BC1
:06011400E05BDFD71200E2
:04011A00C584120086
:10011E00C7B409D01F0EC514016E0150000A03E1C9
:0A012E00010E006E01D0006A1200FD
:10013800086A080E0C6E003408360450085ED8B001
:0E01480002D00826D89000360C2EF5D71200F3
:1001560015C0D9F016C0DAF017C0DBF018C0DCF015
:100166000001D76BD86BD851120802E1D7518E081F
:1001760008E3D2DF005201E004D00001D74BD82BB0
:10018600F2D70001120ED85D02E18F0ED75D03E3B0
:100196007B0E006E24D0C580C5A020D01550161049
:1001A600171018101AE0D951DA11DB11DC110EE123
:1001B60023C0E1FF24C0E2FF050EE66E21C000F079
:1001C60022C001F043DF010E006E09D0010E0001CE
:1001D600D95F000EDA5BDB5BDC5BDED7006A120000
:0C01E60029C000F02AC001F031DF120037
:1001F2000D0E0001E16F17DF0A0E0001E16F13DF40
:020202001200E8
:10020400D7C000F00032009E0032009E0032009EF3
:100214000032009ECD0E0024F66E0C0EF76E000E1A
:10022400F722000EF86E000EF8220900F5CF00F058
:10023400D8C0E1FFD9C0E2FF00C0E6FF010E000113
:10024400D825E16E000ED921E26E0F0ED715006E8F
:10025400CD0E0024F66E0C0EF76E000EF722000E83
:10026400F86E000EF8220900F5CF00F000C0E6FF9A
:10027400020ED825E16E000ED921E26EE66A120064
:100284000001DA6B030EDA5D0AE2DA51D825E16E79
:10029400000ED921E26E200EE66EDA2BF3D7DA5186
:1002A400D825E16E000ED921E26EE66ADA07DA514A
:1002B400D825DB6F000ED921DC6F0A0E046ED7C07F
:1002C40000F038DF08C000F0300E0026DBC0E1FF8C
:1002D400DCC0E2FF00C0E6FF0A0E046ED7C000F0E7
:1002E40029DF00C0D7F00050000A01E102D0DA078C
:0402F400DED712003F
:1002F800D9C0F6FFDAC0F7FFDBC0F8FF0900F5CF79
:1003080000F0005218E0D9C0F6FFDAC0F7FFDBC0F2
:10031800F8FF0900F5CF00F0D7C0E1FFD8C0E2FF31
:1003280000C0E6FF0001D74BD82B010ED927000EDD
:10033800DA23DB23DDD7D7C0E1FFD8C0E2FFE66AC6
:020348001200A1
:10034A00D7C002F0D8C003F002C000F003C001F029
:10035A00024A032A00C0E9FF01C0EAFFEE5201E0A7
:10036A00F3D70001D751025C006ED8510358016ED1
:0A037A00010E005E000E015A120091
:100384000001DA6BD7C0E9FFD8C0EAFFEECFD9F09D
:10039400D951000A0EE0D9C0E1F044DE0001DA2BA5
:1003A400DA51D725E96E000ED821EA6EEECFD9F0E6
:0403B400EFD712006D
:1003B8009E96D7C0C9FF15C0D8F016C0D9F017C08F
:1003C800DAF018C0DBF0C7A421D0155016101710AA
:1003D80018101BE00001D851D911DA11DB110EE118
:1003E80023C0E1FF24C0E2FF040EE66E21C000F046
:1003F80022C001F02ADE010E006E3AD0010E000183
:10040800D85F000ED95BDA5BDB5BDDD715C0D8F0AF
:1004180016C0D9F017C0DAF018C0DBF09EB621D0AC
:1004280015501610171018101BE00001D851D911DB
:10043800DA11DB110EE123C0E1FF24C0E2FF040E54
:10044800E66E21C000F022C001F0FFDD010E006E53
:100458000FD0010E0001D85F000ED95BDA5BDB5BC1
:10046800DDD7C5BC02D0006A03D0C584020E006E79
:02047800120070
:10047A00D7C0F6FFD8C0F7FFD9C0F8FF0900F5CFFB
:10048A00DAF00001DA51000814E2D7C0F6FFD8C04A
:10049A00F7FFD9C0F8FF0900F5CF00F000C0DAF085
:1004AA00010ED727000ED823D92300C0E1F0B7DD0B
:0404BA00E8D712006D
:1004BE00D7C004F0D8C005F004C0E9FF05C0EAFFBC
:1004CE00EE5203E0044A052AF7D704C002F005C035
:1004DE0003F0044A052AD9C000F0DAC001F0000189
:1004EE00D94BDA2B00C0E9FF01C0EAFF02C0E1FFE1
:1004FE0003C0E2FFEECFE6FF02C0E9FF03C0EAFF52
:10050E00EE5201E0E2D7D7C000F0D8C001F01200E1
:10051E00280E0001AB6F000EAC6FE10EAD6F000E3A
:10052E00AE6FFF0EBF6FFF0EC06F000EC16F000EDD
:10053E00C26FFF0EBB6FFF0EBC6F000EBD6F000EC5
:10054E00BE6FFF0EB76FFF0EB86F000EB96F000EC5
:10055E00BA6FAC8A900EAB6E948E949C9EAA03D00A
:08056E00AECF00F0FBD7120034
:10057600806A0F01386B388138833885E70E926EB2
:10058600928A92968096396BFF0E816EFF0E936E5D
:100596009396796A786A8B6A826A3A6B800E946E51
:0405A600606A120075
:1005AA000900F5CFE6FF0006FBE10106F9E11200BA
:1005BA000001D26BD051000825E2A9C0D7F0AAC029
:1005CA00D8F0E80ED96F0C0EDA6F000EDB6F8FDEF3
:1005DA00A9C0D7F0AAC0D8F0B3DECFC0D7F0390E81
:1005EA00D86F000ED96F49DEA9C0D7F0AAC0D8F0DB
:1005FA00390ED96F000EDA6F5DDFA9C0D7F0AAC035
:10060A00D8F0BBDECF51A00AD8B48086C69E9EDD44
:10061A00CFC0D7F0CCDE00C0D1F0000E016EFF0EC5
:10062A00011802E1FF0E001803E1C9CFD1F0C69EFE
:10063A00D5DD80960001D151000A0CE0D26BD05171
:10064A00000807E2DD0ED76F0C0ED86F000ED96FC7
:10065A000FDF40D0010E0001D26F2F0E3724E16E5A
:10066A00000E3820E26ECFC0E6FFD051000830E21B
:10067A00390ED76F000ED86F4A0ED96F0C0EDA6F8B
:10068A00000EDB6F34DE300E3724426ECFC0D7F057
:10069A004E0E0001D86F000ED96FEFDD390ED76FFD
:1006AA00000ED86F6ADEFB0ED76F0C0ED86F000EE5
:1006BA00D96FDEDECFC0D7F0390E0001D86F000E39
:1006CA00D96F9BDD390ED76F000ED86F56DE8CDDE1
:1006DA00374A382A1DDD020E0B6E040E0C6EBA0E56
:1006EA000D6E0D2EFED70C2EFCD70B2EFAD700005E
:1006FA0011DD0050000A01E1FBD70001D0510008CA
:0A070A0001E272DDD2C000F012001F
:10071400CFC015F0D0C016F0D1C017F0D2C018F079
:10072400D3C021F0D4C022F0D5C023F0D6C024F029
:020734001200B1
:100736001E0E0001C36F010EC46F000EC56F000EC2
:10074600C66F560EC76F010EC86F000EC96F000E3A
:10075600CA6F6E0ECB6F000ECC6F000ECD6F000E03
:10076600CE6FFF0EB36FFF0EB46FFF0EB56FFF0EA9
:10077600B66FB80EAF6F030EB06FD70EB16F000E27
:10078600B26F1A0E296E010E2A6E000E2B6E000E27
:100796002C6E949894968B988B9694889486C79E84
:0807A600C79C380EC66E12005C
:1007AE0081EC06F0D38CD38AD388D382D3909B6A04
:1007BE009B9CDADE8096150E0B6E4B0E0C6EBE0EEB
:1007CE000D6E0D2EFED70C2EFCD70B2EFAD7000079
:1007DE002D6A2E6A000E2E5C02E1200E2D5C0AE2BE
:1007EE00390E2D24E16E000E2E20E26EE66A2D4AA1
:1007FE002E2AF0D72D6A2E6A000E2E5C02E1500EC4
:10080E002D5C0AE2590E2D24E16E000E2E20E26EB2
:10081E00E66A2D4A2E2AF0D72D6A2E6A590E00014D
:10082E00A96F000EAA6FB886010EB06EA00EAF6E45
:10083E00AC846EDE0B0E0B6E260E0C6E5D0E0D6E08
:10084E000D2EFED70C2EFCD70B2EFAD70000000073
:10085E000C0EE16F14EC00F00B0E0B6E260E0C6EF0
:10086E005D0E0D6E0D2EFED70C2EFCD70B2EFAD76D
:10087E0000000000B7DC0D0E0001D76F0B0ED86F15
:10088E00000ED96FF3DDEE0E0001D76F0B0ED86F91
:10089E00000ED96FEBDDAA0E0001D76F0C0ED86FCC
:1008AE00000ED96FE3DD9EDC4A0E0001D76F0A0EF3
:1008BE00D86F000ED96FDADD920E0001D76F0A0ED7
:1008CE00D86F000ED96FD2DD680E0001D76F0C0EF7
:1008DE00D86F000ED96FCADD960E0001D76F0C0EC1
:1008EE00D86F000ED96FC2DD7DDC280EC86E1CDFFE
:1008FE00B80ECF6F0B0ED06F000ED16FD26F360EBB
:10090E00D36F000ED46FE10ED56F000ED66FFBDEE7
:10091E008DEC00F08FEC00F00050000A01E1FAD7E8
:10092E00D00E1D6E2D6A2E6A000E2E5C02E1080E90
:10093E002D5C0AE22F0E2D24E16E000E2E20E26EAB
:10094E00E66A2D4A2E2AF0D72D6A2E6A010E1F6EE8
:10095E00000E206E376A386A200E1D6EFE0E1D5C6C
:10096E0022E280BA09D01DC0CFF0010E0001D06F77
:10097E001DDE00C01EF007D01DC0CFF00001D06BF1
:10098E0015DE00C01EF0020E0B6E040E0C6EBA0EBB
:10099E000D6E0D2EFED70C2EFCD70B2EFAD70000A7
:1009AE00020E1D26DBD71EDCB70E0001D76F0B0E15
:1009BE00D86F000ED96F5ADD376A386A000E385C70
:1009CE0002E1080E375C34E2390E0001D76F000EDB
:1009DE00D86FBD0ED96F0C0EDA6F000EDB6F85DC93
:1009EE00310E3724426E2F0E3724E96E000E38205A
:1009FE00EA6EEE50000810E22F0E3724E96E000E5C
:100A0E003820EA6EEECFD7F0460E0001D86F000EFA
:100A1E00D96F02EC01F001D0446A0001390ED76F94
:100A2E00000ED86FA8DCF9EC00F0374A382AC6D78A
:0C0A3E00F9EC00F0D00E1D6EFFD7FFD7C2
:100D020010EE15F0090E006E010E016EF20EF66E77
:0E0D12000C0EF76E000EF86ED5EC02F012001B
:100A4A00204C4344203478323020493243202C2031
:100A5A006D6F64756C652020454570726F6D20322C
:100A6A00344C433235362061766563205254432034
:100A7A0044533133303720737572206C65204275C8
:080A8A0073204932430D0A00FC
:100A9200204176656320522070756C6C2075702041
:100AA200646520322C374B20737572206C6573207D
:100AB2006C69676E65732053434C20657420534400
:100AC200412064752062757320493243200D0A006B
:100AD20020536F75726365203A205F313846323693
:100AE2004B32325F4C6973745F4932435F6465769F
:100AF200696365735F6F6E5F7468655F6275735F6C
:0B0B02003137303833312E630D0A000C
:100B0D00204469726563746F7279203A433A5C5F71
:100B1D004D696B726F435C5F4D657350726F6A65A3
:100B2D0074735F4D696B726F435C5F4C49425F4CF0
:090B3D0043445F4932430D0A00F4
:100B4600204469726563746F7279203A433A5C5F38
:100B56004D696B726F435C5F4D657350726F6A656A
:100B660074735F4D696B726F435C5F4C49425F4CB7
:090B760043445F4932430D0A00BB
:100B7F002050726F6A6574203A5F31384632364BB7
:100B8F0032325F4C6973745F4932435F64657669D3
:100B9F006365735F6F6E5F7468655F6275732E6DEB
:080BAF0063707069200D0A005B
:100BB7004C6973746520646573206164726573732F
:100BC7006573206465206261736520646576696377
:100BD700657320493243206465636F757665727467
:070BE7006573203A0D0A00BE
:100BEE0020536F75726365203A5F31384632364B4B
:100BFE0032325F4C6973745F4932435F6465766964
:100C0E006365735F6F6E5F7468655F6275730D0AFF
:010C1E0000D5
:100C1F00204C6563747572652061647265737365CA
:100C2F00732064657669636520737572206C652027
:0B0C3F0062757320493243200D0A004B
:100C4A0020446576696365202320202066696E64E6
:0E0C5A00206174204020202020202020200037
:100C6800204D6F646520424176617264207369206B
:0A0C7800524135203D30200D0A00E6
:100C8200204D696B726F432070726F20372E3130A6
:040C9200200A0D0027
:100C960020496E697420493243203130304B687ADE
:040CA600200D0A0013
:100CAA002056657273696F6E203A313730383331A6
:030CBA000D0A0020
:100CBD00204465766963652023202020403D200077
:100CCD003031323334353637383941424344454675
:0B0CDD00206E6F7420666F756E64005F
:0A0CE8004465766963652040200032
:040CF20000000000FE
:040CF60000000000FA
:010CFA0000F9
:070CFB0020736F69742000F3
:020000040030CA
:0D00010028193CFFBE81FF0FC00FE00F402B
:0200000400F00A
:1000000028432929207061756C666A756A6F2E66AF
:100010007265652E66720D0A0020202020202020A7
:1000200056657273696F6E2073616E73204C434422
:100030000D0A002020202020202020202020202009
:1000400057726974652054657874206F6E204C4334
:1000500044200D0A002020202020202020202020C5
:100060000000000000000000000000000000000090
:100070000000000000000000000000000000000080
:100080000000000000000000000000000000000070
:100090000000000000000000000000000000000060
:1003E000416D70204F6666733A203531320A0D0038
:1003F0007061756C666A756A6F0A0D000000020E06
:00000001FF
